:0200000480007A
:100000009710000093800000171100001301810277
:1000100083A1000013020000930210001303F0FFFD
:10002000B70300809383F3FF3704008033E241007D
:10003000B3E2510033E36100B3E3710033E48100C4
:100040002320310023224100232451002326610074
:1000500023287100232A8100971000009380C0FAA2
:1000600017110000130181FE03A400009304000097
:10007000130510009305F0FF370600801306F6FF06
:10008000B7060080B36494003365A400B365B40080
:100090003366C400B366D40023208100232291007C
:1000A0002324A1002326B1002328C100232AD10044
:1000B00097100000938080F517110000130181FA5A
:1000C00083A6000013070000930710001308F0FF39
:1000D000B70800809388F8FF3709008033E7E6000F
:1000E000B3E7F60033E80601B3E8160133E9260169
:1000F0002320D1002322E1002324F1002326010143
:1001000023281101232A210197100000938040F039
:1001100017110000130181F603A9000093090000E4
:10012000130A1000930AF0FF370B0080130BFBFF3C
:10013000B70B0080B3693901336A4901B36A5901C9
:10014000336B6901B36B7901232021012322310133
:10015000232441012326510123286101232A71010F
:1001600097100000938000EB17110000130181F23B
:1001700083AB0000130C0000930C1000130DF0FF74
:10018000B70D0080938DFDFF370E008033EC8B019F
:10019000B3EC9B0133EDAB01B3EDBB0133EECB010F
:1001A0002320710123228101232491012326A1010F
:1001B0002328B101232AC101971C0000938CCCE5B0
:1001C000171D0000130D8DEE03AE0C00130200018D
:1001D00093020002130300049303000813040010A9
:1001E00093040080B36E4E0033EF5E00B36F6F0078
:1001F000B3E07F0033E18000B361910023204D0024
:100200002322CD012324DD012326ED012328FD0136
:10021000232A1D00232C2D00232E3D0097100000C3
:100220009380C0DF17110000130141EA03AE000004
:10023000B79DFFF7938D8D813360BE0123200100B0
:10024000971000009380C0DD17110000130141E8F2
:1002500003AE0000B79DFFF7938D8D813360BE0123
:10026000B3620000232001002322510097100000F8
:10027000938040DB17110000130101E683A1000009
:1002800033E20100B36202003363500033670300BE
:10029000B367070033E80700B36C0001336D9001CA
:1002A000B36D0D00232041002322A1012324B101BD
:1002B00017150000130505D897150000938585E2F2
:1002C000370610F01306C6F26306B5028326C50092
:1002D0002320D600832685002320D60083264500D0
:1002E0002320D600832605002320D6001305050110
:1002F0006FF09FFD370510F0130505F22320050070
:0403000000000000F9
:101000000000000001000000FFFFFFFFFFFFFF7F67
:10101000000000800D0000007856341298BADCFE03
:10102000145892360000000000000000000000008C
:10103000FFFFFFFFFFFFFFFFFFFFFFFFFFFFFFFFC0
:10104000FFFFFFFFFFFFFFFFFFFFFFFFFFFFFFFFB0
:10105000FFFFFFFFFFFFFFFFFFFFFFFFFFFFFFFFA0
:10106000FFFFFFFFFFFFFFFFFFFFFFFFFFFFFFFF90
:10107000FFFFFFFFFFFFFFFFFFFFFFFFFFFFFFFF80
:10108000FFFFFFFFFFFFFFFFFFFFFFFFFFFFFFFF70
:10109000FFFFFFFFFFFFFFFFFFFFFFFFFFFFFFFF60
:1010A000FFFFFFFFFFFFFFFFFFFFFFFFFFFFFFFF50
:1010B000FFFFFFFFFFFFFFFFFFFFFFFFFFFFFFFF40
:1010C000FFFFFFFFFFFFFFFFFFFFFFFFFFFFFFFF30
:1010D000FFFFFFFFFFFFFFFFFFFFFFFFFFFFFFFF20
:040000058000000077
:00000001FF
